:1000000000C008E107BB06E108BB0FED0DBF882467
:10001000112743D0E02E77D0B19B0FC0B29B03C015
:10002000B09B06C0F9CFC49A3ED0C4984BD0F4CF51
:10003000C49A3BD0C49846D0EFCF5DD059D0B29B84
:1000400015C0B09B08C0B19901C0F8CF57D0112797
:100050000E2D1CD0E1CFE3940E2D0A3118F009E1EA
:10006000E02E0BC050D01FD02DD0EDCFEE2029F0C8
:10007000EA9449D018D026D0E6CF04E62CD000E58B
:1000800023D004E628D00AEF1FD0DDCFE199FECFC0
:100090000DBB1EBBE29AE19A0895E199FECF1EBB0B
:1000A000E09A0DB3089511E001C013E00F2DC3983D
:1000B0001CD0C39A1AD00A95D1F71A95B9F70895AA
:1000C00012E001C011E00F2D13D00A95E9F71A953F
:1000D00008950F2D000FC39805D0C39A03D00A9539
:1000E000D1F70895E2E3F0E00BC0EDE7F0E008C0DF
:1000F000EAEFF0E005C0E4ECF9E002C0E8E8F3E183
:100100003197F1F70895E4E1F1E0EE0DF81DC8959F
:10011000F02C08951E1F202122232425262728297C
:0E0120002A2B2C2D2E3032373C41465064786D
:00000001FF
